:1000000022C046C045C044C043C0B0C341C040C088
:100010003FC03EC03DC03CC03BC03AC039C00000FC
:10002000000038000000000037000000000036002B
:10003000020202020202020202020102040810206D
:10004000200410089F0611241FBECFE5D2E0DEBFBA
:10005000CDBF10E0A0E6B0E0EEEAFEE002C0059001
:100060000D92A437B107D9F721E0A4E7B0E001C0B1
:100070001D92A736B207E1F710E0C3E2D0E003C05B
:100080002197FE0108D7C232D107D1F7B9D30DC7E6
:10009000B7CFDF92EF92FF920F931F93CF93DF932F
:1000A000962F282F30E0EE24E394822F203408F09E
:1000B0006CC08901B3E015950795BA95E1F7422F19
:1000C0004770DE2C01C0DD0C4A95EAF7E0E1F1E073
:1000D000DF0158E0F12C60E041E0792F742359F002
:1000E0001996CD91DC911A97C00FD11F7A817D218D
:1000F00009F446C0642B440F515012965111EDCFB4
:10010000FF2009F43FC06623E9F1C0E0248D2F3FB2
:1001100029F0CF5F3496CF30C9F7C0E00C2F10E044
:10012000F801EE0FFF1FEE0FFF1FE45DFE4F80830F
:1001300020E0492F50E090FD07C055954795942F3A
:100140002F5F2830B1F720E0000F111F000F111FA3
:10015000005F1E4FF801238FD1E0D80F8D2F99DF5C
:10016000F801868F6F2D8D2F94DFF801858F8C2FEE
:10017000DF91CF911F910F91FF90EF90DF90089545
:10018000F42AB9CF2F5F3F4F90CFE0E1F1E0C0E01C
:10019000848D8F3F29F0CF5F3496CF30C9F7C0E010
:1001A000EC2FF0E0DF01AA0FBB1FAA0FBB1FA45D5D
:1001B000BE4F80E88C9380E0692F70E090FD07C00F
:1001C00075956795962F8F5F8830B1F780E0EE0FB9
:1001D000FF1FEE0FFF1FE05FFE4F838F8FEF868FB5
:1001E000C5CF282FFC01842F9191892798E03CE806
:1001F000869508F483279A95D9F79E2F921B961718
:1002000098F30895FC01A381B481828130E020E05D
:100210009C91982349F42F5F3F4F23353105C1F757
:100220008FE0808381E0089530E020E09C91982366
:1002300041F02F5F3F4F2E3094E23907B9F788E045
:10024000F0CF4CE050E060E070E09C91982329F4FE
:100250004150510961097109C1F781E0452B462BD5
:10026000472B09F780E00895AF92BF92CF92DF92BB
:10027000EF92FF920F931F93CF93DF93EC01C42E65
:10028000F894EB81FC8192818A8180958923828315
:10029000EB81FC8191818A818095892381838B0107
:1002A000E12C88E0A82EB12CFF24F394D12CCE01B0
:1002B000A9DF8111DF2888818823A1F091E0F9125C
:1002C00004C0883011F48EE08883789481E0DF9157
:1002D000CF911F910F91FF90EF90DF90CF90BF9043
:1002E000AF900895FF0CE1E0AE1AB10801F7F801F4
:1002F000D1928F01E394CE10D4CF789480E0E7CFF1
:10030000FC01A381B481828130E020E09C9198239C
:1003100049F42F5F3F4F23353105C1F78FE08083CC
:1003200081E0089530E020E09C91982369F02F5FF0
:100330003F4F2E3094E23907B9F788E0F0CF44E21E
:1003400050E060E070E00CC06111F9CF11969C9113
:100350001197892B11968C9342E150E060E070E098
:10036000A381B48182819C91982329F44150510941
:1003700061097109C1F711969C91119780958923A4
:1003800011968C9380E00895AF92BF92CF92DF9246
:10039000EF92FF920F931F93CF93DF93EC01E42E24
:1003A000F894EB81FC8192818A81809589238283F4
:1003B000EB81FC8191818A81809589238183B62E8E
:1003C0008B01F801A1908F0188E0C82ED12CFF2469
:1003D000F39461E08A2D8F2109F460E0CE0190DF73
:1003E0008823A1F0F1E0FF1205C09881983011F444
:1003F0009EE098837894DF91CF911F910F91FF90A9
:10040000EF90DF90CF90BF90AF900895FF0C81E008
:10041000C81AD108F1F6902F9B199E1590F2789486
:1004200081E0E912E8CF80E0E6CFE62FF0E025E0BA
:10043000F595E7952A95E1F7E43060F4E80FF91FA8
:10044000E557FF4F8081809529F06F718295880F65
:10045000807E682B862F08957F928F929F92AF9215
:10046000BF92CF92DF92EF92FF920F931F93CF93A1
:10047000DF9300D000D000D0CDB7DEB77C018B0178
:100480001E8241E0BE016C5F7F4FC801EDDE81112D
:10049000D7C04E8161E0CE010496A3DE8E8342E098
:1004A000BE016F5F7F4FC801DFDE8111C9C04E8181
:1004B00062E0CE01019695DE8E838A818111C0C0F3
:1004C0008C818A3A09F40AC108F085C08F3009F09E
:1004D00046C0470122E9820E911C67013AE8C30E2B
:1004E000D11CAA24A394B12C9981F401808198177E
:1004F00008F0A6C041E0BE016B5F7F4FC801B4DECB
:1005000081119EC04E8161E0CE0105966ADE8E8328
:1005100041E0BE016A5F7F4FC80136DF811190C0A4
:100520007980672DC70181DFF3E0F71550F0F60100
:100530004081950101C0220F7A94EAF7242309F043
:10054000F1C01B8241E0BE016D5F7F4FC8011CDF1F
:10055000811176C089818F5F89838E83C5CF853570
:1005600009F0FEC08981883008F06AC041E0BE0110
:100570006B5F7F4FC80178DE811162C04E8161E000
:10058000CE0105962EDE8E8341E0BE016A5F7F4F6D
:10059000C801FADE811154C02981C701820F911D63
:1005A000253038F4FC01E657FF4F2D81308123239D
:1005B000208386579F4FFC0180818D8341E0BE01DF
:1005C0006B5F7F4FC801E0DE81113AC089818F5F88
:1005D00089838E83C7CF833C09F446C0803F09F0EE
:1005E000BFC041E0BE016A5F7F4FC801CDDE81110F
:1005F00027C01E829980570182E9A80EB11CF5011F
:1006000080819816B8F4692DC7010FDFC82ED12C50
:10061000FAE0CF0ED11CCE0CDF1C41E0B601C801C0
:10062000B3DE81110DC04E8161E0C601DADD8E833B
:100630009394E5CF41E0BE016A5F7F4FC801A4DE1D
:1006400026960FB6F894DEBF0FBECDBFDF91CF91D7
:100650001F910F91FF90EF90DF90CF90BF90AF90E0
:100660009F908F907F90089541E0BE016A5F7F4F19
:10067000C8018ADE8111E4CF570122E9A20EB11C24
:100680009980F50180819816D8F61E82892D807E8A
:1006900090E2892E880E9814B8F4692DC701C5DE42
:1006A000C82ED12CFAE0CF0ED11CCE0CDF1C41E0BD
:1006B000B601C80169DE8111C3CF4E8161E0C60178
:1006C00090DD8E839394E7CF41E0BE016A5F7F4F58
:1006D000C8015ADE8111B4CF8982D2CF41E0BE0178
:1006E0006A5F7F4FC80150DE8111AACF1E82D98078
:1006F000ED0CF11C27E02D1508F49CCF57013AE8CA
:10070000A30EB11C41E0B501C8013EDE9FEFE91A1E
:10071000F90A811195CF4E8161E0C50162DD8E83BA
:10072000D394E8CF682F70E0F701E60FF71F9285AA
:100730002D8192239287843068F4CB010496950131
:1007400002C0220F331F8A95E2F7C90180958423E6
:10075000F6018083665F7F4F6E0D7F1D41E0F6CE10
:100760009BE0F801908381836BCF9BD31F920F9204
:100770000FB60F9211242F933F938F939F93AF93B4
:10078000BF938091790090917A00A0917B00B09105
:100790007C003091780026E0230F2D3758F5029623
:1007A000A11DB11D209378008093790090937A0069
:1007B000A0937B00B0937C008091740090917500B1
:1007C000A0917600B09177000196A11DB11D809394
:1007D000740090937500A0937600B0937700BF915A
:1007E000AF919F918F913F912F910F900FBE0F90DE
:1007F0001F90189529E8230F0396A11DB11DD2CF94
:10080000CF93DF93CDB7DEB729970FB6F894DEBF4D
:100810000FBECDBF78948AB582608ABD8AB58160EB
:100820008ABD83B7826083BF83B7816083BF89B786
:10083000826089BF80B7826080BF80B7816080BFDF
:10084000329A319A3098379A8CB580648CBD8091F9
:100850001801883008F03FC0A9E1B1E09D017FEFA9
:1008600090E0F901419151919F01F0E04D375F0710
:1008700091F1793018F0452B09F4792F9F5F98306A
:1008800081F77F3F41F1E72FF0E0EE0FFF1FE05FC0
:10089000FE4F2DE730E0328721878F5F809318016C
:1008A000E0E1F1E029E231E081E060E04D915D912D
:1008B000452B09F0682B880F2A173B07B9F78CE402
:1008C00091E02FEF248F34968E179F07D9F7662378
:1008D00011F080E0DEDBECE6F0E0AFE8B0E084E7CA
:1008E00090E021912D938E179F07D9F780910701F2
:1008F0008F7E8093070101E010E010921001FF2429
:10090000F39480911801882309F450C0E0911301F9
:10091000F091140191818091120180958923818346
:1009200090911001E0911301F09114018091120156
:100930009F3091F41092100141E950E060E070E0C6
:100940009081982329F44150510961097109C1F737
:10095000452B462B472B89F19081982339F144E0B0
:100960005CE060E070E09081982329F041505109EB
:1009700061097109C1F7452B462B472BB9F04EE4AD
:1009800052E060E070E09081982329F441505109D1
:1009900061097109C1F7411551056105710509F436
:1009A00091C0473451406105710598F080E090E0B6
:1009B000892B09F4A2CF24DBA0CF4EE452E060E003
:1009C00070E09081982329F441505109610971091F
:1009D000C1F74CE050E060E070E09081982329F08E
:1009E0004150510961097109C1F7928180958923AC
:1009F0008283E0911301F0911401818190911201A1
:100A0000892B8183E0911301F0911401209112014F
:100A100030E082E690E0A0E0B0E00097A105B105EB
:100A200081F04081422351E009F450E0531304C0A7
:100A30000197A109B109A9F73F250097A105B105C3
:100A400061F7818120952823218385EC90E0A0E047
:100A5000B0E0E0911301F091140130911201208176
:100A6000232321F40197A109B109C9F7892B8A2B06
:100A70008B2B61F141E0BE01675F7F4F80E191E028
:100A8000F3DB809110018F3009F43BCF81118ECFC1
:100A90008985893611F108F04EC0833309F42CC1E1
:100AA000B8F48F3009F428C19AE090931001809334
:100AB0001101809110018F3009F423CF882309F4AC
:100AC00020CF74CF84E08093100170CF86E0FBCFFD
:100AD0008C3309F4ECC0853539F710922A01109255
:100AE000290148E0BE016F5F7F4F80E191E0BCDBF0
:100AF0008111DFCF89E1C82E81E0D82ED6018D91FA
:100B00009D916D01009709F4CBC0DC0112969E0106
:100B10002F5F3F4FAC01465F5F4F7D91F9016191BF
:100B20009F017613BDC0A417B507B9F790932A01AA
:100B300080932901D7C08C3C09F4B9C058F4853A98
:100B400009F0B2CF8091290190912A01009709F014
:100B5000C9C02CCF8C3E09F4ACCF803F09F0A4CFA4
:100B600010922A0110922901B0902B01A0902C0123
:100B7000F894D12CC12CE12CAC1050C060E080E185
:100B800091E0BEDB8111BDCE60E080E191E0B8DB99
:100B90008111B7CE80E191E035DB90911001911188
:100BA000B0CE2E2D30E0220F331F220F331F205FD7
:100BB0003E4F882381F1D9015E96EC908E2D90E016
:100BC000FC01EE0FFF1FEE0FFF1FE05FFE4FB38C27
:100BD000FFEFAA24AA94EF1641F0880F991F880FFF
:100BE000991FFC01E45DFE4FA0802FEFC21AD20ACC
:100BF00060E4C616D10409F0BFCF7894EB2DF0E085
:100C0000EE0FFF1FE05FFE4F8185928590932A01D2
:100C10008093290176CEF901E58CD0CFEB2DF0E061
:100C2000EE0FFF1FE05FFE4F0184F285E02DC6014D
:100C300033E0959587953A95E1F7E80FF91F8C2DEC
:100C40008770980101C0220F8A95EAF7828182237A
:100C5000C9F061E080E191E053DB811152CE60E0A8
:100C600080E191E04DDB81114CCE9924939480E199
:100C700091E0C8DA90911001911143CE891509F4E1
:100C8000B4CF3FCE60E080E191E03ADB811139CE14
:100C900061E080E191E034DB982E882341F331CE8E
:100CA000F9E2CF16F1E0DF0609F028CF7FCE809180
:100CB000290190912A01892B71F4809118018130CA
:100CC00051F4E9E1F1E0819191910097E1F3909382
:100CD0002A01809329018091290190912A0100978E
:100CE00009F40FCEDC01ED91FC910190F081E02D33
:100CF00060E171E00995DDCE8091290190912A0192
:100D0000892B71F480911801813051F4E9E1F1E00F
:100D1000819191910097E1F390932A0180932901A9
:100D20006091290170912A016115710509F4E9CDDD
:100D30006E5F7F4F48E080E191E026DBE2CDCF930C
:100D4000DF93109210011092180110922A01109254
:100D5000290110921A011092190110921C0110928F
:100D60001B0110921E0110921D0110922001109281
:100D70001F01109222011092210110922401109261
:100D80002301109226011092250110922801109241
:100D900027012AE330E0F90184918093120180E376
:100DA00090E0FC014491E42FF0E0EE0FFF1FE65DC0
:100DB000FF4F459154915093140140931301F90151
:100DC0002491FC0184918823B9F090E0880F991F49
:100DD000FC01EC5DFF4FC591D491FC01E25EFF4F39
:100DE000A591B4919FB7F894888120958223888338
:100DF0008C9128232C939FBFE0911301F091140153
:100E000092818091120180958923828384E690E00B
:100E100090937E0080937D008AEB80937F008CE02E
:100E20008093800084E8809381008FE28093820029
:100E300080E58093830085E08093840080E1809347
:100E4000850040E067E08FE790E0CBD98093860093
:100E50008AE690E090937E0080937D00E7E8F0E0E2
:100E600090E08FEF81939F5F9038E1F780930701C7
:100E7000809308018093090180930A0180930B01FC
:100E800080930C0180930D0110920E0190930F013D
:100E9000DF91CF910895EE0FFF1F0590F491E02DA3
:0E0EA000099481E090E0F89400C0F894FFCF30
:100EAE0000000000B503000000002C025210055097
:040EBE002F840CBAB7
:00000001FF
